:020000040000FA
:04080000F2EF07F01C
:1008100003B213EF05F0F2B431EF05F09EB039EFFB
:1008200005F09EB241EF05F0F2A81AEF04F0F2B223
:1008300025EF04F0F2A620EF04F0F2B022EF04F06E
:10084000A1EF07F0F296F290FF00CD90F2929EA0F9
:100850002FEF04F00101533F2FEF04F0542BAEC1F2
:10086000B2F1AFC1B3F1B0C1B4F1B1C1B5F1AAC138
:10087000AEF1ABC1AFF1ACC1B0F1ADC1B1F1A6C148
:10088000AAF1A7C1ABF1A8C1ACF1A9C1ADF1A2C158
:10089000A6F1A3C1A7F1A4C1A8F1A5C1A9F19EC168
:1008A000A2F19FC1A3F1A0C1A4F1A1C1A5F19AC178
:1008B0009EF19BC19FF19CC1A0F19DC1A1F196C188
:1008C0009AF197C19BF198C19CF199C19DF1CECF4E
:1008D00096F1CFCF97F153C198F154C199F1CF6AF6
:1008E000CE6A0101536B546B9E90CD800FBC0F8E6E
:1008F0000FBA7EEF04F00F8AA1EF07F00F8C0FBE46
:10090000BAEF04F096C19AF197C19BF198C19CF19E
:1009100099C19DF19AC19EF19BC19FF19CC1A0F12B
:100920009DC1A1F19EC1A2F19FC1A3F1A0C1A4F1FB
:10093000A1C1A5F1A2C1A6F1A3C1A7F1A4C1A8F1CB
:10094000A5C1A9F1A6C1AAF1A7C1ABF1A8C1ACF19B
:10095000A9C1ADF1AAC1AEF1ABC1AFF1ACC1B0F16B
:10096000ADC1B1F1AEC1B2F1AFC1B3F1B0C1B4F13B
:10097000B1C1B5F101015E6B5F6B606B616B96514C
:100980005E2797515F2398516023995161239A51B3
:100990005E279B515F239C5160239D5161239E5193
:1009A0005E279F515F23A0516023A1516123A25173
:1009B0005E27A3515F23A4516023A5516123A65153
:1009C0005E27A7515F23A8516023A9516123AA5133
:1009D0005E27AB515F23AC516023AD516123AE5113
:1009E0005E27AF515F23B0516023B1516123B251F3
:1009F0005E27B3515F23B4516023B5516123D89072
:100A00000101613360335F335E33D890010161339C
:100A100060335F335E33D8900101613360335F33FD
:100A20005E33A1EF07F00392ABB2AB98AB88030142
:100A300003EE00F080517F0BE92604C0EFFF802B0E
:100A40008151805D700BD8A48B8200008051815D44
:100A5000700BD8A48B9281518019D8B40790A1EF64
:100A600007F0F2940101453FA1EF07F0462BA1EFFB
:100A700007F09E900101533FA1EF07F0542BA1EF27
:100A800007F09E92040062A146EF05F0077C07ACD8
:100A900061EF05F0C274C2B45BEF05F0C3CFB3F5EC
:100AA000C4CFB4F50501D890B433B333D890B43380
:100AB000B33362EF05F0C3CF55F1C4CF56F162EF07
:100AC00005F0C28207B4CFEF05F047C14BF148C132
:100AD0004CF149C14DF14AC14EF15EC162F15FC1B5
:100AE00063F160C164F161C165F196C1B6F197C16E
:100AF000B7F198C1B8F199C1B9F19AC1BAF19BC1E6
:100B0000BBF19CC1BCF19DC1BDF19EC1BEF19FC1B5
:100B1000BFF1A0C1C0F1A1C1C1F1A2C1C2F1A3C185
:100B2000C3F1A4C1C4F1A5C1C5F1A6C1C6F1A7C155
:100B3000C7F1A8C1C8F1A9C1C9F1AAC1CAF1ABC125
:100B4000CBF1ACC1CCF1ADC1CDF1AEC1CEF1AFC1F5
:100B5000CFF1B0C1D0F1B1C1D1F1B2C1D2F1B3C1C5
:100B6000D3F1B4C1D4F1B5C1D5F1B3C5B5F5B4C5B0
:100B7000B6F5B5C5B7F5B6C5B8F5010155515B2752
:100B800056515C23E86A5D230E2ECFEF05F05CC161
:100B900057F15DC158F15B6B5C6B5D6B078E0201B9
:100BA000002FA1EF07F03C0E006F00C10CF101C156
:100BB0000DF102C10EF103C10FF104C110F105C125
:100BC00011F106C112F107C113F108C114F109C1F5
:100BD00015F10AC116F10BC117F134C135F1050148
:100BE0002F51000AD8B4A0EF06F005012F51010AD9
:100BF000D8B42AEF06F005012F51020AD8B46BEFE2
:100C000006F005012F51030AD8B46BEF06F0050179
:100C10002F51040AD8B46BEF06F005012F51050AD5
:100C2000D8B46BEF06F005012F51060AD8B46BEF6C
:100C300006F005012F51070AD8B46BEF06F0050145
:100C40002F51320AD8B428EF06F02F6BA0EF06F030
:100C5000A0EF06F00501536735EF06F0546735EF56
:100C600006F0556735EF06F0566739EF06F0A0EF4E
:100C700006F057C500F158C501F159C502F15AC532
:100C800003F10101010E046F000E056F000E066FE7
:100C9000000E076FF3EC1FF000C157F501C158F5C6
:100CA00002C159F503C15AF500675EEF06F001670E
:100CB0005EEF06F002675EEF06F00367A0EF06F056
:100CC00053C557F554C558F555C559F556C55AF588
:100CD0000F88A0EF06F00501306771EF06F0A0EF76
:100CE00006F00FBE86EF06F010A08BEF06F00101B4
:100CF000476782EF06F0486782EF06F0496782EFA8
:100D000006F04A6786EF06F08BEF06F007AE8BEF32
:100D100006F09DEF06F00501312FA0EF06F03C0E26
:100D2000316F302FA0EF06F00101000E626FE00E70
:100D3000636FA50E646F010E656F0501306B0F8840
:100D40000501626B33B7A6EF06F062810CC100F1BA
:100D50000DC101F10EC102F10FC103F110C104F187
:100D600011C105F112C106F113C107F114C108F157
:100D700015C109F116C10AF117C10BF135C134F1E2
:100D800000C10CF101C10DF102C10EF103C10FF15F
:100D900004C110F105C111F106C112F107C113F12F
:100DA00008C114F109C115F10AC116F10BC117F1FF
:100DB00034C135F101018A67E5EF06F08B67E5EF95
:100DC00006F08C67E5EF06F08D67E9EF06F019EFA6
:100DD00007F08EC100F18FC101F190C102F191C104
:100DE00003F10101010E046F000E056F000E066F86
:100DF000000E076FF3EC1FF000C18EF101C18FF1FF
:100E000002C190F103C191F100670EEF07F0016795
:100E10000EEF07F002670EEF07F0036719EF07F018
:100E20008AC18EF18BC18FF18CC190F18DC191F18E
:100E30000F80D57ED5BE69D0D6CF47F1D7CF48F148
:100E400045C149F1E86AE8CF4AF1109047C100F185
:100E500048C101F149C102F14AC103F101010A0E81
:100E6000046F000E056F000E066F000E076FF3ECA7
:100E70001FF003AF1080010154A74BEF07F00F9A4A
:100E80000F9C0F9E0101000E5E6F600E5F6F3D0EA6
:100E9000606F080E616F010147BF5BEF07F04867A5
:100EA0005BEF07F049675BEF07F04A675BEF07F01E
:100EB000F28880EF07F0F2985E6B5F6B606B616B9E
:100EC000966B976B986B996B9A6B9B6B9C6B9D6BFE
:100ED0009E6B9F6BA06BA16BA26BA36BA46BA56BAE
:100EE000A66BA76BA86BA96BAA6BAB6BAC6BAD6B5E
:100EF000AE6BAF6BB06BB16BB26BB36BB46BB56B0E
:100F0000D76AD66A0101456B466B0CC100F10DC171
:100F100001F10EC102F10FC103F110C104F111C1C1
:100F200005F112C106F113C107F114C108F115C191
:100F300009F116C10AF117C10BF135C134F1A1EF66
:100F400007F002C0E0FF005001C0D8FF1000A6B2B9
:100F5000A7EF07F00CC0A9FF0BC0A8FFA69EA69C98
:100F6000A684F29E550EA76EAA0EA76EA682F28EDA
:100F7000A694A6B2B9EF07F00C2A1200A96EA69E9D
:100F8000A69CA680A8500C2A120004012C0E826F89
:100F9000B6EC0AF0EEEC20F00C50BEEC07F0E8CF17
:100FA00000F10C50BEEC07F0E8CF01F101AFDEEF2D
:100FB00007F00101FF0E026FFF0E036F91EC20F0AE
:100FC0002967EAEF07F00401200E826FB6EC0AF001
:100FD000EFEF07F004012D0E826FB6EC0AF0BBECC8
:100FE0001EF01200076A0F6A106A0F010D0EC16E23
:100FF000860EC06E030EC26E0F01680E896E130E50
:10100000926E080E8A6EF30E936E8B6A900E946E3B
:10101000F18EF19E0E6A01015B6B5C6B5D6B576B31
:10102000586BF29A0101476B486B496B4A6B4B6BEB
:101030004C6B4D6B4E6B4F6B506B516B526B456BEA
:10104000466BD76AD66A0F01280ED56EF28A9D903C
:10105000B00ECD6E01015E6B5F6B606B616B626B9E
:10106000636B646B656B666B676B686B696B536B0B
:10107000546BCF6ACE6A0F9A0F9C0F9E9D80760E9E
:10108000CA6E9D8202013C0E006FCC6A160EBEEC49
:1010900007F0E8CF00F1170EBEEC07F0E8CF01F142
:1010A000180EBEEC07F0E8CF02F1190EBEEC07F007
:1010B000E8CF03F1010103AF78EF08F0EEEC20F088
:1010C000160E0C6E00C10BF0A7EC07F0170E0C6E9D
:1010D00001C10BF0A7EC07F0180E0C6E02C10BF06B
:1010E000A7EC07F0190E0C6E03C10BF0A7EC07F08C
:1010F00000C18AF101C18BF102C18CF103C18DF1F4
:1011000000C18EF101C18FF102C190F103C191F1D3
:101110001A0EBEEC07F0E8CF00F11B0EBEEC07F094
:10112000E8CF01F11C0EBEEC07F0E8CF02F11D0E76
:10113000BEEC07F0E8CF03F1010103AFCEEF08F0FA
:10114000EEEC20F01A0E0C6E00C10BF0A7EC07F0CD
:101150001B0E0C6E01C10BF0A7EC07F01C0E0C6E01
:1011600002C10BF0A7EC07F01D0E0C6E03C10BF0D3
:10117000A7EC07F01A0EBEEC07F0E8CF00F11B0E4B
:10118000BEEC07F0E8CF01F11C0EBEEC07F0E8CF93
:1011900002F11D0EBEEC07F0E8CF03F100C192F1A1
:1011A00001C193F102C194F103C195F1240EAC6E1B
:1011B000900EAB6E240EAC6E080EB86E000EB06EC4
:1011C0001F0EAF6E0401806B816B0F01900EAB6E32
:1011D0000F019D8A0301806B816BC26B8B9234EC93
:1011E00026F034EC26F090EC27F013EC24F0200EDF
:1011F000BEEC07F0E8CF2FF505012F51FF0AD8A468
:1012000009EF09F02F6B200E0C6E2FC50BF0A7EC29
:1012100007F00501010E306F3C0E316F250EBEEC5C
:1012200007F0E8CF00F1260EBEEC07F0E8CF01F1A1
:10123000270EBEEC07F0E8CF02F1280EBEEC07F057
:10124000E8CF03F1010103AF40EF09F0EEEC20F02D
:10125000250E0C6E00C10BF0A7EC07F0260E0C6EED
:1012600001C10BF0A7EC07F0270E0C6E02C10BF0CA
:10127000A7EC07F0280E0C6E03C10BF0A7EC07F0EB
:1012800000C153F501C154F502C155F503C156F52E
:1012900000C157F501C158F502C159F503C15AF50E
:1012A000290EBEEC07F0E8CF5BF505015C515B5DF4
:1012B000D8A05BC55CF505012F51020A0EE181B88B
:1012C0006DEF09F005015C2F6AEF09F05BC55CF575
:1012D0006DEF09F081BACFEF27F0210EBEEC07F0D9
:1012E000E8CF00F1220EBEEC07F0E8CF01F1230EAB
:1012F000BEEC07F0E8CF02F1240EBEEC07F0E8CF19
:1013000003F1010103AFB3EF09F0EEEC20F0210E81
:101310000C6E00C10BF0A7EC07F0220E0C6E01C1A1
:101320000BF0A7EC07F0230E0C6E02C10BF0A7EC3C
:1013300007F0240E0C6E03C10BF0A7EC07F0210E92
:10134000BEEC07F0E8CF00F1220EBEEC07F0E8CFCC
:1013500001F1230EBEEC07F0E8CF02F1240EBEEC43
:1013600007F0E8CF03F100C15DF501C15EF502C1F0
:101370005FF503C160F54AEC23F00CEC22F05CEC65
:1013800021F005012F51030A12E005012F51040A33
:101390001DE005012F51050A24E005012F51060A21
:1013A00032E005012F51070A38E016EF0AF0ACC50C
:1013B00000F101010F0E001701010051000A36E093
:1013C00001010051050A32E013EF0AF0ACC500F14B
:1013D00001010F0E001701010051000A27E013EF71
:1013E0000AF00501AC51000A21E00501AC51150AD3
:1013F0001DE00501AC51300A19E00501AC51450A68
:1014000015E013EF0AF00501AC51000A0FE00501E9
:10141000AC51300A0BE013EF0AF00501AC51000AA1
:1014200005E013EF0AF081BACFEF27F00790000133
:10143000F28EF28C07B03CEF1DF00FB01BEF18F0EE
:101440000FB8DFEF11F00301805181197F0BD8B481
:101450003CEF1DF013EE00F081517F0BE126812B54
:10146000E7CFE8FFE00BD8B43CEF1DF023EE82F0AD
:10147000C2513F0BD926E7CFDFFFC22BDF50780ADE
:10148000D8A43CEF1DF007808EC100F18FC101F19F
:1014900090C102F191C103F10101040E046F000E2D
:1014A000056F000E066F000E076FF3EC1FF000AF24
:1014B00063EF0AF00101030E8E6F000E8F6F000EB6
:1014C000906F000E916F03018251720AD8B41BEF26
:1014D00018F08251520AD8B41BEF18F08251750AE5
:1014E000D8B41BEF18F08251630AD8B4F6EF19F0A4
:1014F0008251690AD8B4D6EF14F082517A0AD8B46E
:10150000E9EF15F08251490AD8B475EF14F0825111
:10151000500AD8B493EF13F08251700AD8B4D6EFC2
:1015200013F08251540AD8B401EF14F08251740AB6
:10153000D8B447EF14F082516D0AD8B4CAEF0AF05C
:1015400082514D0AD8B4E3EF0AF08251730AD8B43D
:101550004BEF17F08251530AD8B4B0EF17F0825115
:101560004C0AD8B472EF0BF02DEF1AF0040114EE10
:1015700000F080517F0BE12682C4E7FF802B120030
:1015800004010D0E826FB6EC0AF00A0E826FB6EC03
:101590000AF0120004016D0E826FB6EC0AF003012E
:1015A0008351300AD8B422EF0BF003018351310A82
:1015B000D8B435EF0BF003018351320AD8B448EFA9
:1015C0000BF02DEF1AF004014D0E826FB6EC0AF00D
:1015D0002FEC21F084C331F185C332F186C333F19E
:1015E0000101296B3CEC21F0B3EC20F003018351A5
:1015F000300AD8B40AEF0BF003018351310AD8B492
:1016000012EF0BF003018351320AD8B41AEF0BF03A
:101610002DEF1AF0FD0E0C6E00C10BF0A7EC07F0D9
:1016200022EF0BF0FE0E0C6E00C10BF0A7EC07F0E2
:1016300035EF0BF0FF0E0C6E00C10BF0A7EC07F0BE
:1016400048EF0BF00401300E826FB6EC0AF0040193
:101650002C0E826FB6EC0AF0EEEC20F0FD0EBEEC24
:1016600007F0E8CF00F159EF0BF00401310E826F63
:10167000B6EC0AF004012C0E826FB6EC0AF0EEEC28
:1016800020F0FE0EBEEC07F0E8CF00F159EF0BF0B2
:101690000401320E826FB6EC0AF0EEEC20F0040189
:1016A0002C0E826FB6EC0AF0FF0EBEEC07F0E8CF0E
:1016B00000F191EC20F031C182F40401300E822758
:1016C000B6EC0AF032C182F40401300E8227B6EC87
:1016D0000AF033C182F40401300E8227B6EC0AF01E
:1016E0002BEF1AF003018351300AD8B4D7EF0EF074
:1016F00003018351310AD8B4E5EF0FF003018351A0
:10170000320AD8B453EF10F003018351330AD8B42E
:1017100063EF10F003018351340AD8B473EF10F073
:1017200003018351350AD8B4E4EF11F0030183516A
:10173000360AD8B412EF12F003018351370AD8B435
:1017400039EF0EF003018351460AD8B438EF11F097
:10175000030183514D0AD8B4B2EF0CF00301835159
:101760006D0AD8B4CCEF0CF0030183515A0AD8B4F7
:101770005FEF0FF003018351490AD8B412EF13F061
:1017800003018351500AD8B444EF12F0030183518E
:10179000540AD8B4BDEF12F003018351630AD8B4E0
:1017A000ECEF0CF003018351430AD8B4E4EF0DF0E1
:1017B00003018351730AD8B4EAEF0CF0030183519B
:1017C000610AD8B4FFEF0BF003018351650AD8B466
:1017D00027EF0FF003018351450AD8B435EF0FF01E
:1017E00003018351620AD8B443EF0FF00301835120
:1017F000420AD8B451EF0FF0D8A42DEF1AF004012B
:101800004C0E826FB6EC0AF00401610E826FB6ECEA
:101810000AF00CEC22F004012C0E826FB6EC0AF0F8
:10182000EEEC20F0ABC500F1010191EC20F031C1EC
:1018300082F40401300E8227B6EC0AF032C182F441
:101840000401300E8227B6EC0AF033C182F40401A1
:10185000300E8227B6EC0AF004012C0E826FB6EC33
:101860000AF0EEEC20F0ACC500F1010191EC20F0A3
:1018700031C182F40401300E8227B6EC0AF032C185
:1018800082F40401300E8227B6EC0AF033C182F4F0
:101890000401300E8227B6EC0AF004012C0E826F90
:1018A000B6EC0AF0EEEC20F0ADC500F1010191ECD0
:1018B00020F031C182F40401300E8227B6EC0AF028
:1018C00032C182F40401300E8227B6EC0AF033C133
:1018D00082F40401300E8227B6EC0AF004012C0ECB
:1018E000826FB6EC0AF0EEEC20F0AEC500F101011B
:1018F00091EC20F031C182F40401300E8227B6EC65
:101900000AF032C182F40401300E8227B6EC0AF0EC
:1019100033C182F40401300E8227B6EC0AF00401D0
:101920002C0E826FB6EC0AF0EEEC20F0B3C500F19D
:10193000010191EC20F031C182F40401300E8227C4
:10194000B6EC0AF032C182F40401300E8227B6EC04
:101950000AF033C182F40401300E8227B6EC0AF09B
:1019600040EF12F02FEC21F084C333F13CEC21F076
:10197000B3EC20F0200E0C6E00C10BF0A7EC07F0CA
:1019800000C12FF505012F51000A06E005012F5176
:10199000010A02E0B2EC22F004014C0E826FB6ECB8
:1019A0000AF004014D0E826FB6EC0AF004012C0E11
:1019B000826FB6EC0AF0EEEC20F02FC500F191EC4E
:1019C00020F033C182F40401300E8227B6EC0AF015
:1019D00040EF12F0CFEF27F004014C0E826FB6EC0F
:1019E0000AF00401630E826FB6EC0AF05CEC21F0A1
:1019F00004012C0E826FB6EC0AF001EC0DF040EF02
:101A000012F0EEEC20F0B1C500F10101003B0F0E29
:101A1000001791EC20F033C182F40401300E8227CC
:101A2000B6EC0AF0B1C500F101010F0E010100177B
:101A300091EC20F033C182F40401300E8227B6EC21
:101A40000AF004012D0E826FB6EC0AF0B0C500F169
:101A50000101003B0F0E001791EC20F033C182F41E
:101A60000401300E8227B6EC0AF0B0C500F1010186
:101A70000F0E0101001791EC20F033C182F4040134
:101A8000300E8227B6EC0AF004012D0E826FB6EC00
:101A90000AF0AFC500F10101003B0F0E001791ECF9
:101AA00020F033C182F40401300E8227B6EC0AF034
:101AB000AFC500F101010F0E0101001791EC20F0FC
:101AC00033C182F40401300E8227B6EC0AF004011F
:101AD000200E826FB6EC0AF0AEC500F10F0E0101C8
:101AE000001791EC20F033C182F40401300E8227FC
:101AF000B6EC0AF00401200E826FB6EC0AF0ADC518
:101B000000F101010101003B0F0E001791EC20F0E4
:101B100033C182F40401300E8227B6EC0AF0ADC561
:101B200000F101010F0E0101001791EC20F033C10B
:101B300082F40401300E8227B6EC0AF004013A0E5A
:101B4000826FB6EC0AF0ACC500F10101003B0F0E4C
:101B5000001791EC20F033C182F40401300E82278B
:101B6000B6EC0AF0ACC500F101010F0E010100173F
:101B700091EC20F033C182F40401300E8227B6ECE0
:101B80000AF004013A0E826FB6EC0AF0ABC500F120
:101B90000101003B0F0E001791EC20F033C182F4DD
:101BA0000401300E8227B6EC0AF0ABC500F101014A
:101BB0000F0E001791EC20F033C182F40401300EB7
:101BC0008227B6EC0AF0120084C3E8FF0F0BE83A54
:101BD000E8CFB1F585C3E8FF0F0B0501B11387C34B
:101BE000E8FF0F0BE83AE8CFB0F588C3E8FF0F0B2A
:101BF0000501B0138AC3E8FF0F0BE83AE8CFAFF551
:101C00008BC3E8FF0F0B0501AF138DC3E8FF0F0B6C
:101C1000E8CFAEF58FC3E8FF0F0BE83AE8CFADF59C
:101C200090C3E8FF0F0B0501AD1392C3E8FF0F0B44
:101C3000E83AE8CFACF593C3E8FF0F0B0501AC130E
:101C400095C3E8FF0F0BE83AE8CFABF596C3E8FF82
:101C50000F0B0501AB13BBEC21F004014C0E826F9E
:101C6000B6EC0AF00401430E826FB6EC0AF0F6EF10
:101C70000CF0078404014C0E826FB6EC0AF00401EC
:101C8000370E826FB6EC0AF004012C0E826FB6ECB0
:101C90000AF005012E51130A06E005012E51170A1C
:101CA0000DE0D4EF0EF00101000E006F000E016F89
:101CB000100E026F000E036F67EF0EF00101000EB1
:101CC000006F000E016F000E026F010E036F91ECAA
:101CD00020F02AC182F40401300E8227B6EC0AF00B
:101CE0002BC182F40401300E8227B6EC0AF02CC11D
:101CF00082F40401300E8227B6EC0AF02DC182F482
:101D00000401300E8227B6EC0AF02EC182F40401E1
:101D1000300E8227B6EC0AF02FC182F40401300E97
:101D20008227B6EC0AF030C182F40401300E82271B
:101D3000B6EC0AF031C182F40401300E8227B6EC11
:101D40000AF032C182F40401300E8227B6EC0AF0A8
:101D500033C182F40401300E8227B6EC0AF004018C
:101D60002C0E826FB6EC0AF00101100E006F000E0F
:101D7000016F000E026F000E036F91EC20F031C175
:101D800082F40401300E8227B6EC0AF032C182F4EC
:101D90000401300E8227B6EC0AF033C182F404014C
:101DA000300E8227B6EC0AF0079440EF12F0078459
:101DB00090EC27F0EEEC20F02DC500F191EC20F036
:101DC00004014C0E826FB6EC0AF00401300E826FF3
:101DD000B6EC0AF004012C0E826FB6EC0AF031C1A9
:101DE00082F40401300E8227B6EC0AF032C182F48C
:101DF0000401300E8227B6EC0AF033C182F40401EC
:101E0000300E8227B6EC0AF004012C0E826FB6EC7D
:101E10000AF0EEEC20F02EC500F191EC20F031C17B
:101E200082F40401300E8227B6EC0AF032C182F44B
:101E30000401300E8227B6EC0AF033C182F40401AB
:101E4000300E8227B6EC0AF0079440EF12F004013E
:101E50004C0E826FB6EC0AF00401650E826FB6EC90
:101E60000AF09BEC23F040EF12F004014C0E826F5D
:101E7000B6EC0AF00401450E826FB6EC0AF0B8EC3D
:101E800023F040EF12F004014C0E826FB6EC0AF022
:101E90000401620E826FB6EC0AF0F2EC23F040EF20
:101EA00012F004014C0E826FB6EC0AF00401420EEF
:101EB000826FB6EC0AF0D5EC23F040EF12F004018B
:101EC0004C0E826FB6EC0AF004015A0E826FB6EC2B
:101ED0000AF004012C0E826FB6EC0AF090EC27F0A9
:101EE000EEEC20F005012E51130A06E005012E51FB
:101EF000170A0DE090EF0FF00101000E006F000EC9
:101F0000016F100E026F000E036F90EF0FF00101D2
:101F1000000E006F000E016F000E026F010E036FC6
:101F20000101100E046F000E056F000E066F000E0B
:101F3000076F24EC20F091EC20F02AC182F4040118
:101F4000300E8227B6EC0AF02BC182F40401300E69
:101F50008227B6EC0AF02CC182F40401300E8227ED
:101F6000B6EC0AF02DC182F40401300E8227B6ECE3
:101F70000AF02EC182F40401300E8227B6EC0AF07A
:101F80002FC182F40401300E8227B6EC0AF030C172
:101F900082F40401300E8227B6EC0AF031C182F4DB
:101FA0000401300E8227B6EC0AF032C182F404013B
:101FB000300E8227B6EC0AF033C182F40401300EF1
:101FC0008227B6EC0AF040EF12F0078404014C0EB1
:101FD000826FB6EC0AF00401310E826FB6EC0AF0A3
:101FE00004012C0E826FB6EC0AF025C500F126C55F
:101FF00001F127C502F128C503F10101100E046F9C
:10200000000E056F000E066F000E076F24EC20F027
:1020100091EC20F02AC182F40401300E8227B6EC44
:102020000AF02BC182F40401300E8227B6EC0AF0CC
:102030002CC182F40401300E8227B6EC0AF02DC1C7
:1020400082F40401300E8227B6EC0AF02EC182F42D
:102050000401300E8227B6EC0AF02FC182F404018D
:10206000300E8227B6EC0AF030C182F40401300E43
:102070008227B6EC0AF031C182F40401300E8227C7
:10208000B6EC0AF032C182F40401300E8227B6ECBD
:102090000AF033C182F40401300E8227B6EC0AF054
:1020A000079440EF12F0078404014C0E826FB6ECE7
:1020B0000AF00401320E826FB6EC0AF0EAEC25F069
:1020C000079440EF12F0078404014C0E826FB6ECC7
:1020D0000AF00401330E826FB6EC0AF047EC26F0EA
:1020E0000794F0EF0FF0078404014C0E826FB6ECFA
:1020F0000AF00401340E826FB6EC0AF004012C0ED3
:10210000826FB6EC0AF02FEC21F084C32AF185C36C
:102110002BF186C32CF187C32DF188C32EF189C31F
:102120002FF18AC330F18BC331F18CC332F18DC3EF
:1021300033F10101296B3CEC21F0B3EC20F0100EDF
:10214000046F000E056F000E066F000E076F04ECA3
:1021500020F000C121F501C122F502C123F503C120
:1021600024F543EC27F034C5ABF535C5ACF536C5E1
:10217000ADF537C5AEF538C5AFF539C5B0F53AC5DB
:10218000B1F501EC0DF004012C0E826FB6EC0AF0F3
:102190003BC500F13CC501F13DC502F13EC503F16F
:1021A0000101000E046F000E056F010E066F000E98
:1021B000076F24EC20F091EC20F02967E2EF10F09B
:1021C000E7EF10F004012D0E826FB6EC0AF030C17B
:1021D00082F40401300E8227B6EC0AF031C182F499
:1021E0000401300E8227B6EC0AF004012E0E826F35
:1021F000B6EC0AF032C182F40401300E8227B6EC4C
:102200000AF033C182F40401300E8227B6EC0AF0E2
:1022100004012C0E826FB6EC0AF0EEEC20F03FC504
:1022200000F140C501F157EC1BF004012C0E826F48
:10223000B6EC0AF0EEEC20F041C500F191EC20F094
:1022400031C182F40401300E8227B6EC0AF032C1AB
:1022500082F40401300E8227B6EC0AF033C182F416
:102260000401300E8227B6EC0AF0079440EF12F01A
:102270002FEC21F085C32AF186C32BF187C32CF103
:1022800088C32DF189C32EF18AC32FF18BC330F19E
:102290008CC331F18DC332F18EC333F10101296B4F
:1022A0003CEC21F0B3EC20F00101010E046F000EB4
:1022B000056F000E066F000E076FF3EC1FF0100E97
:1022C000046F000E056F000E066F000E076F04EC22
:1022D00020F000C129F501C12AF502C12BF503C187
:1022E0002CF571EC25F004014C0E826FB6EC0AF06F
:1022F0000401460E826FB6EC0AF004012C0E826FC8
:10230000B6EC0AF025C500F126C501F127C502F19A
:1023100028C503F10101100E046F000E056F000EB9
:10232000066F000E076F24EC20F091EC20F02AC11C
:1023300082F40401300E8227B6EC0AF02BC182F43D
:102340000401300E8227B6EC0AF02CC182F404019D
:10235000300E8227B6EC0AF02DC182F40401300E53
:102360008227B6EC0AF02EC182F40401300E8227D7
:10237000B6EC0AF02FC182F40401300E8227B6ECCD
:102380000AF030C182F40401300E8227B6EC0AF064
:1023900031C182F40401300E8227B6EC0AF032C15A
:1023A00082F40401300E8227B6EC0AF033C182F4C5
:1023B0000401300E8227B6EC0AF040EF12F00F98BD
:1023C00047EC26F02DEF1AF004014C0E826FB6ECAC
:1023D0000AF00401350E826FB6EC0AF004012C0EEF
:1023E000826FB6EC0AF0EEEC20F00784B5C500F180
:1023F000079491EC20F031C182F40401300E822761
:10240000B6EC0AF032C182F40401300E8227B6EC39
:102410000AF033C182F40401300E8227B6EC0AF0D0
:1024200040EF12F00AEC26F0EEEC20F033C500F19C
:1024300091EC20F004014C0E826FB6EC0AF004011E
:10244000360E826FB6EC0AF004012C0E826FB6ECE9
:102450000AF031C182F40401300E8227B6EC0AF092
:1024600032C182F40401300E8227B6EC0AF033C187
:1024700082F40401300E8227B6EC0AF040EF12F02D
:10248000C0EC0AF02DEF1AF004014C0E826FB6EC8E
:102490000AF00401500E826FB6EC0AF004012C0E13
:1024A000826FB6EC0AF085C32AF186C32BF187C38D
:1024B0002CF188C32DF189C32EF18AC32FF18BC370
:1024C00030F18CC331F18DC332F18EC333F1010190
:1024D0003CEC21F0B3EC20F003018451530A0DE0F1
:1024E000030184514D0A38E00401780E826FB6EC86
:1024F0000AF0C0EC0AF02DEF1AF00401530E826FBF
:10250000B6EC0AF0250E0C6E00C10BF0A7EC07F03C
:10251000260E0C6E01C10BF0A7EC07F0270E0C6E17
:1025200002C10BF0A7EC07F0280E0C6E03C10BF0F4
:10253000A7EC07F000C153F501C154F502C155F5F0
:1025400003C156F500C157F501C158F502C159F54F
:1025500003C15AF521EF13F004014D0E826FB6EC62
:102560000AF0290E0C6E00C10BF0A7EC07F000C1B9
:102570005BF500C15CF521EF13F004014C0E826F96
:10258000B6EC0AF00401540E826FB6EC0AF00401B6
:102590002C0E826FB6EC0AF084C32AF185C32BF1AE
:1025A00086C32CF187C32DF188C32EF189C32FF187
:1025B0008AC330F18BC331F18DC332F18EC333F155
:1025C00001013CEC21F0B3EC20F00101000E046F9E
:1025D000000E056F010E066F000E076F04EC20F071
:1025E000210E0C6E00C10BF0A7EC07F0220E0C6E52
:1025F00001C10BF0A7EC07F0230E0C6E02C10BF02B
:10260000A7EC07F0240E0C6E03C10BF0A7EC07F04B
:1026100000C15DF501C15EF502C15FF503C160F562
:1026200021EF13F004014C0E826FB6EC0AF00401A6
:10263000490E826FB6EC0AF004012C0E826FB6ECE4
:102640000AF0250EBEEC07F0E8CF00F1260EBEEC36
:1026500007F0E8CF01F1270EBEEC07F0E8CF02F15A
:10266000280EBEEC07F0E8CF03F191EC20F074ECFB
:102670001EF00401730E826FB6EC0AF004012C0EFA
:10268000826FB6EC0AF0EEEC20F0290EBEEC07F0FB
:10269000E8CF00F191EC20F074EC1EF00401730E11
:1026A000826FB6EC0AF004012C0E826FB6EC0AF0D1
:1026B00057C500F158C501F159C502F15AC503F1DA
:1026C00091EC20F074EC1EF00401730E826FB6ECF6
:1026D0000AF004012C0E826FB6EC0AF0EEEC20F04A
:1026E0005CC500F191EC20F074EC1EF004016D0E5D
:1026F000826FB6EC0AF004012C0E826FB6EC0AF081
:102700005DC500F15EC501F15FC502F160C503F171
:1027100048EC1AF004012C0E826FB6EC0AF0C0EC03
:102720000AF02DEF1AF083C32AF184C32BF185C37D
:102730002CF186C32DF187C32EF188C32FF189C3F5
:1027400030F18AC331F18BC332F18CC333F1010113
:102750003CEC21F0B3EC20F0160E0C6E00C10BF037
:10276000A7EC07F0170E0C6E01C10BF0A7EC07F0F9
:10277000180E0C6E02C10BF0A7EC07F0190E0C6ED0
:1027800003C10BF0A7EC07F000C18AF101C18BF186
:1027900002C18CF103C18DF100C18EF101C18FF135
:1027A00002C190F103C191F175EF14F083C32AF1D6
:1027B00084C32BF185C32CF186C32DF187C32EF181
:1027C00088C32FF189C330F18AC331F18BC332F151
:1027D0008CC333F101013CEC21F0B3EC20F000C1DB
:1027E0008AF101C18BF102C18CF103C18DF100C1ED
:1027F0008EF101C18FF102C190F103C191F175EF2A
:1028000014F083C32AF184C32BF185C32CF186C352
:102810002DF187C32EF188C32FF189C330F18AC30C
:1028200031F18CC332F18DC333F101013CEC21F065
:10283000B3EC20F00101000E046F000E056F010ED5
:10284000066F000E076F04EC20F01A0E0C6E00C12C
:102850000BF0A7EC07F01B0E0C6E01C10BF0A7EC00
:1028600007F01C0E0C6E02C10BF0A7EC07F01D0E5A
:102870000C6E03C10BF0A7EC07F000C192F101C18F
:1028800093F102C194F103C195F175EF14F083C384
:102890002AF184C32BF185C32CF186C32DF187C3A4
:1028A0002EF188C32FF189C330F18AC331F18CC373
:1028B00032F18DC333F101013CEC21F0B3EC20F097
:1028C0000101000E046F000E056F010E066F000E71
:1028D000076F04EC20F000C192F101C193F102C135
:1028E00094F103C195F175EF14F0160EBEEC07F0EC
:1028F000E8CF00F1170EBEEC07F0E8CF01F1180E9B
:10290000BEEC07F0E8CF02F1190EBEEC07F0E8CFFD
:1029100003F191EC20F074EC1EF00401730E826F51
:10292000B6EC0AF004012C0E826FB6EC0AF08AC1F4
:1029300000F18BC101F18CC102F18DC103F191EC69
:1029400020F074EC1EF00401730E826FB6EC0AF0F6
:1029500004012C0E826FB6EC0AF01A0EBEEC07F0E2
:10296000E8CF00F11B0EBEEC07F0E8CF01F11C0E22
:10297000BEEC07F0E8CF02F11D0EBEEC07F0E8CF89
:1029800003F148EC1AF004012C0E826FB6EC0AF049
:1029900092C100F193C101F194C102F195C103F11B
:1029A00048EC1AF0C0EC0AF02DEF1AF00401690EA1
:1029B000826FB6EC0AF004012C0E826FB6EC0AF0BE
:1029C0000101040E006F000E016F000E026F000E79
:1029D000036F91EC20F02CC182F40401300E8227A9
:1029E000B6EC0AF02DC182F40401300E8227B6EC59
:1029F0000AF02EC182F40401300E8227B6EC0AF0F0
:102A00002FC182F40401300E8227B6EC0AF030C1E7
:102A100082F40401300E8227B6EC0AF031C182F450
:102A20000401300E8227B6EC0AF032C182F40401B0
:102A3000300E8227B6EC0AF033C182F40401300E66
:102A40008227B6EC0AF004012C0E826FB6EC0AF075
:102A50000101060E006F000E016F000E026F000EE6
:102A6000036F91EC20F02CC182F40401300E822718
:102A7000B6EC0AF02DC182F40401300E8227B6ECC8
:102A80000AF02EC182F40401300E8227B6EC0AF05F
:102A90002FC182F40401300E8227B6EC0AF030C157
:102AA00082F40401300E8227B6EC0AF031C182F4C0
:102AB0000401300E8227B6EC0AF032C182F4040120
:102AC000300E8227B6EC0AF033C182F40401300ED6
:102AD0008227B6EC0AF004012C0E826FB6EC0AF0E5
:102AE0000101240E006F000E016F000E026F000E38
:102AF000036F91EC20F02CC182F40401300E822788
:102B0000B6EC0AF02DC182F40401300E8227B6EC37
:102B10000AF02EC182F40401300E8227B6EC0AF0CE
:102B20002FC182F40401300E8227B6EC0AF030C1C6
:102B300082F40401300E8227B6EC0AF031C182F42F
:102B40000401300E8227B6EC0AF032C182F404018F
:102B5000300E8227B6EC0AF033C182F40401300E45
:102B60008227B6EC0AF004012C0E826FB6EC0AF054
:102B7000200EF86EF76AF66A04010900F5CF82F4B8
:102B8000B6EC0AF00900F5CF82F4B6EC0AF00900C1
:102B9000F5CF82F4B6EC0AF00900F5CF82F4B6EC7A
:102BA0000AF00900F5CF82F4B6EC0AF00900F5CF7F
:102BB00082F4B6EC0AF00900F5CF82F4B6EC0AF024
:102BC0000900F5CF82F4B6EC0AF0C0EC0AF02DEF64
:102BD0001AF08351630AD8A42DEF1AF08451610AC8
:102BE000D8A42DEF1AF085516C0AD8A42DEF1AF055
:102BF0008651410A42E08651440A1BE08651420A4E
:102C0000D8B450EF16F08651350AD8B4B7EF1BF0A0
:102C10008651360AD8B40CEF1CF08651370AD8B466
:102C200075EF1CF08651380AD8B4D3EF1CF02DEFA5
:102C30001AF00798079A04017A0E826FB6EC0AF030
:102C40000401780E826FB6EC0AF00401640E826F04
:102C5000B6EC0AF081A834EF16F00401550E826F2D
:102C6000B6EC0AF039EF16F004014C0E826FB6ECA8
:102C70000AF0C0EC0AF02DEF1AF00788079A040159
:102C80007A0E826FB6EC0AF00401410E826FB6EC48
:102C90000AF00401610E826FB6EC0AF02AEF16F01A
:102CA0000798078A04017A0E826FB6EC0AF00401D5
:102CB000420E826FB6EC0AF00401610E826FB6EC30
:102CC0000AF02AEF16F0010166676EEF16F06767EB
:102CD0006EEF16F068676EEF16F0696786EF16F014
:102CE0004F677AEF16F050677AEF16F051677AEF78
:102CF00016F0526786EF16F00101000E006F000E0D
:102D0000016F000E026F000E036F12000101620ED0
:102D1000046F010E056F000E066F000E076F66C18F
:102D200000F167C101F168C102F169C103F1F3EC7F
:102D30001FF003BF0AEF17F00101000E046FA80E89
:102D4000056F550E066F020E076F66C100F167C171
:102D500001F168C102F169C103F166C186F167C181
:102D600087F168C188F169C189F1F3EC1FF003BFF5
:102D7000C3EF16F00101000E866FA80E876F550E87
:102D8000886F020E896F0E0EBEEC07F0E8CF18F1C7
:102D90000F0EBEEC07F0E8CF19F1100EBEEC07F0F5
:102DA000E8CF1AF1110EBEEC07F0E8CF1BF13CECB6
:102DB0001FF086C104F187C105F188C106F189C100
:102DC00007F1F3EC1FF0078200EC1FF03CEC1FF062
:102DD000079200EC1FF086C100F187C101F188C1A4
:102DE00002F189C103F1079200EC1FF0CC0E046FD1
:102DF000E00E056F870E066F050E076FF3EC1FF0F0
:102E000000C118F101C119F102C11AF103C11BF18E
:102E100042EF17F00101800E006F1A0E016F060ECF
:102E2000026F000E036F4FC104F150C105F151C193
:102E300006F152C107F1F3EC1FF003AF23EF17F0D7
:102E4000EEEC20F012000E0EBEEC07F0E8CF18F109
:102E50000F0EBEEC07F0E8CF19F1100EBEEC07F034
:102E6000E8CF1AF1110EBEEC07F0E8CF1BF14FC10D
:102E700000F150C101F151C102F152C103F10782C9
:102E800000EC1FF018C100F119C101F11AC102F1E3
:102E90001BC103F112000401730E826FB6EC0AF03D
:102EA00004012C0E826FB6EC0AF0078462C166F151
:102EB00063C167F164C168F165C169F14BC14FF14C
:102EC0004CC150F14DC151F14EC152F157C159F1B0
:102ED00058C15AF1079471EC17F0C0EC0AF02DEFCD
:102EE0001AF066C100F167C101F168C102F169C160
:102EF00003F1010191EC20F074EC1EF00401630E6B
:102F0000826FB6EC0AF004012C0E826FB6EC0AF068
:102F10004FC100F150C101F151C102F152C103F1A1
:102F2000010191EC20F074EC1EF00401660E826F3A
:102F3000B6EC0AF004012C0E826FB6EC0AF0EEEC4F
:102F400020F059C100F15AC101F1010191EC20F0CA
:102F500074EC1EF00401740E826FB6EC0AF01200DD
:102F600010820401530E826FB6EC0AF004012C0E9D
:102F7000826FB6EC0AF083C32AF184C32BF185C3B8
:102F80002CF186C32DF187C32EF188C32FF189C39D
:102F900030F18AC331F18BC332F18CC333F10101BB
:102FA0003CEC21F0B3EC20F000C166F101C167F107
:102FB00002C168F103C169F18EC32AF18FC32BF1FD
:102FC00090C32CF191C32DF192C32EF193C32FF135
:102FD00094C330F195C331F196C332F197C333F105
:102FE00001013CEC21F0B3EC20F000C14FF101C134
:102FF00050F102C151F103C152F12FEC21F099C3FC
:103000002FF19AC330F19BC331F19CC332F19DC3C0
:1030100033F101013CEC21F0B3EC20F000C159F197
:1030200001C15AF171EC17F004012C0E826FB6EC5D
:103030000AF022EF18F08251520A03E10F8222EFC8
:1030400018F00F928251750A03E1108429EF18F0ED
:1030500010948251550A03E1108630EF18F0109653
:10306000078410B28DEF18F010A479EF18F0B6C1F4
:1030700066F1B7C167F1B8C168F1B9C169F1BAC108
:103080006AF1BBC16BF1BCC16CF1BDC16DF1BEC1D8
:103090006EF1BFC16FF1C0C170F1C1C171F1C2C1A8
:1030A00072F1C3C173F1C4C174F1C5C175F1C6C178
:1030B00076F1C7C177F1C8C178F1C9C179F1CAC148
:1030C0007AF1CBC17BF1CCC17CF1CDC17DF1CEC118
:1030D0007EF1CFC17FF1D0C180F1D1C181F1D2C1E8
:1030E00082F1D3C183F1D4C184F1D5C185F181EFDF
:1030F00018F062C166F163C167F164C168F165C12E
:1031000069F14BC14FF14CC150F14DC151F14EC16C
:1031100052F157C159F158C15AF107940FA0AFEFBE
:1031200018F0010192679CEF18F093679CEF18F07C
:1031300094679CEF18F09567A0EF18F0AFEF18F0C8
:1031400063EC16F092C104F193C105F194C106F14C
:1031500095C107F1F3EC1FF003BFF3EF19F063EC37
:1031600016F00101000E046F000E056F010E066FD0
:10317000000E076F24EC20F010A4C6EF18F0040135
:10318000750E826FB6EC0AF0CBEF18F00401720EE8
:10319000826FB6EC0AF004012C0E826FB6EC0AF0D6
:1031A00091EC20F02967DAEF18F00401200E826F0D
:1031B000DDEF18F004012D0E826FB6EC0AF030C17D
:1031C00082F40401300E8227B6EC0AF031C182F499
:1031D0000401300E8227B6EC0AF004012E0E826F35
:1031E000B6EC0AF032C182F40401300E8227B6EC4C
:1031F0000AF033C182F40401300E8227B6EC0AF0E3
:1032000004016D0E826FB6EC0AF004012C0E826F81
:10321000B6EC0AF04FC100F150C101F151C102F109
:1032200052C103F1010191EC20F074EC1EF0040195
:10323000480E826FB6EC0AF004017A0E826FB6EC8B
:103240000AF004012C0E826FB6EC0AF066C100F1A0
:1032500067C101F168C102F169C103F1010191EC9B
:1032600020F074EC1EF00401630E826FB6EC0AF0DD
:1032700004012C0E826FB6EC0AF066C100F167C142
:1032800001F168C102F169C103F101010A0E046F85
:10329000000E056F000E066F000E076F04EC20F0A5
:1032A000000E046F120E056F000E066F000E076F02
:1032B00024EC20F091EC20F02AC182F40401300EBD
:1032C0008227B6EC0AF02BC182F40401300E82276B
:1032D000B6EC0AF02CC182F40401300E8227B6EC61
:1032E0000AF02DC182F40401300E8227B6EC0AF0F8
:1032F0002EC182F40401300E8227B6EC0AF02FC1F1
:1033000082F40401300E8227B6EC0AF030C182F458
:103310000401300E8227B6EC0AF004012E0E826FF3
:10332000B6EC0AF031C182F40401300E8227B6EC0B
:103330000AF032C182F40401300E8227B6EC0AF0A2
:1033400033C182F40401300E8227B6EC0AF0040186
:10335000730E826FB6EC0AF004012C0E826FB6EC8D
:103360000AF0EEEC20F059C100F15AC101F157EC1E
:103370001BF00FB2BFEF19F00FA0F1EF19F004012D
:103380002C0E826FB6EC0AF0200EF86EF76AF66A21
:1033900004010900F5CF82F4B6EC0AF00900F5CF7C
:1033A00082F4B6EC0AF00900F5CF82F4B6EC0AF02C
:1033B0000900F5CF82F4B6EC0AF00900F5CF82F4EB
:1033C000B6EC0AF00900F5CF82F4B6EC0AF0090079
:1033D000F5CF82F4B6EC0AF00900F5CF82F4B6EC32
:1033E0000AF0C0EC0AF00F902DEF1AF00401630E02
:1033F000826FB6EC0AF004012C0E826FB6EC0AF074
:1034000033EC1AF004012C0E826FB6EC0AF0A6EC35
:103410001AF004012C0E826FB6EC0AF022EC1BF0BD
:1034200004012C0E826FB6EC0AF00101F80E006F59
:10343000CD0E016F660E026F030E036F48EC1AF09B
:1034400004012C0E826FB6EC0AF038EC1BF0C0ECD5
:103450000AF02DEF1AF0C0EC0AF00301C26B0790DE
:1034600010923CEF1DF0D8900E0EBEEC07F0E8CFA6
:1034700000F10F0EBEEC07F0E8CF01F1100EBEEC2C
:1034800007F0E8CF02F1110EBEEC07F0E8CF03F130
:103490000101000E046F000E056F010E066F000E95
:1034A000076F24EC20F091EC20F02AC182F4040193
:1034B000300E8227B6EC0AF02BC182F40401300EE4
:1034C0008227B6EC0AF02CC182F40401300E822768
:1034D000B6EC0AF02DC182F40401300E8227B6EC5E
:1034E0000AF02EC182F40401300E8227B6EC0AF0F5
:1034F0002FC182F40401300E8227B6EC0AF030C1ED
:1035000082F40401300E8227B6EC0AF031C182F455
:103510000401300E8227B6EC0AF004012E0E826FF1
:10352000B6EC0AF032C182F40401300E8227B6EC08
:103530000AF033C182F40401300E8227B6EC0AF09F
:1035400004016D0E826FB6EC0AF01200120EBEEC92
:1035500007F0E8CF00F1130EBEEC07F0E8CF01F161
:10356000140EBEEC07F0E8CF02F1150EBEEC07F02A
:10357000E8CF03F101010A0E046F000E056F000E83
:10358000066F000E076F04EC20F0000E046F120EA1
:10359000056F000E066F000E076F24EC20F091EC13
:1035A00020F02AC182F40401300E8227B6EC0AF022
:1035B0002BC182F40401300E8227B6EC0AF02CC134
:1035C00082F40401300E8227B6EC0AF02DC182F499
:1035D0000401300E8227B6EC0AF02EC182F40401F9
:1035E000300E8227B6EC0AF02FC182F40401300EAF
:1035F0008227B6EC0AF030C182F40401300E822733
:10360000B6EC0AF004012E0E826FB6EC0AF031C15E
:1036100082F40401300E8227B6EC0AF032C182F443
:103620000401300E8227B6EC0AF033C182F40401A3
:10363000300E8227B6EC0AF00401730E826FB6ECEE
:103640000AF012000A0EBEEC07F0E8CF00F10B0EF4
:10365000BEEC07F0E8CF01F10C0EBEEC07F0E8CFAE
:1036600002F10D0EBEEC07F0E8CF03F157EF1BF0AF
:10367000060EBEEC07F0E8CF00F1070EBEEC07F037
:10368000E8CF01F1080EBEEC07F0E8CF02F1090E19
:10369000BEEC07F0E8CF03F157EF1BF00101EEECB1
:1036A00020F0078457C100F158C101F107940101CE
:1036B000E80E046F800E056F000E066F000E076F98
:1036C00004EC20F0000E046F040E056F000E066F70
:1036D000000E076F24EC20F0880E046F130E056FA8
:1036E000000E066F000E076FF3EC1FF00A0E046F5A
:1036F000000E056F000E066F000E076F24EC20F021
:1037000091EC20F0010129678BEF1BF00401200EE2
:10371000826F8EEF1BF004012D0E826FB6EC0AF063
:1037200030C182F40401300E8227B6EC0AF031C1B8
:1037300082F40401300E8227B6EC0AF032C182F422
:103740000401300E8227B6EC0AF004012E0E826FBF
:10375000B6EC0AF033C182F40401300E8227B6ECD5
:103760000AF00401430E826FB6EC0AF0120087C320
:103770002AF188C32BF189C32CF18AC32DF18BC3A5
:103780002EF18CC32FF18DC330F18EC331F190C374
:1037900032F191C333F10101296B3CEC21F0B3EC20
:1037A00020F00101000E046F000E056F010E066F80
:1037B000000E076F04EC20F00E0E0C6E00C10BF033
:1037C000A7EC07F00F0E0C6E01C10BF0A7EC07F091
:1037D000100E0C6E02C10BF0A7EC07F0110E0C6E70
:1037E00003C10BF0A7EC07F004017A0E826FB6EC70
:1037F0000AF004012C0E826FB6EC0AF00401350EBB
:10380000826FB6EC0AF004012C0E826FB6EC0AF05F
:1038100033EC1AF039EF16F087C32AF188C32BF185
:1038200089C32CF18AC32DF18BC32EF18CC32FF1E8
:103830008DC330F18EC331F190C332F191C333F1B6
:103840000101296B3CEC21F0B3EC20F0880E046FF1
:10385000130E056F000E066F000E076FF8EC1FF0D9
:10386000000E046F040E056F000E066F000E076F4A
:1038700004EC20F00101E80E046F800E056F000ECD
:10388000066F000E076F24EC20F00A0E0C6E00C1CC
:103890000BF0A7EC07F00B0E0C6E01C10BF0A7ECC0
:1038A00007F00C0E0C6E02C10BF0A7EC07F00D0E2A
:1038B0000C6E03C10BF0A7EC07F004017A0E826FC7
:1038C000B6EC0AF004012C0E826FB6EC0AF004018B
:1038D000360E826FB6EC0AF004012C0E826FB6EC45
:1038E0000AF022EC1BF039EF16F087C32AF188C3E7
:1038F0002BF189C32CF18AC32DF18BC32EF18CC31C
:103900002FF18DC330F18FC331F190C332F191C3E8
:1039100033F101013CEC21F0B3EC20F0000E046F18
:10392000120E056F000E066F000E076F04EC20F0FC
:1039300001010A0E046F000E056F000E066F000EE7
:10394000076F24EC20F0120E0C6E00C10BF0A7ECF8
:1039500007F0130E0C6E01C10BF0A7EC07F0140E6C
:103960000C6E02C10BF0A7EC07F0150E0C6E03C134
:103970000BF0A7EC07F004017A0E826FB6EC0AF0A8
:1039800004012C0E826FB6EC0AF00401370E826F30
:10399000B6EC0AF004012C0E826FB6EC0AF0A6EC2D
:1039A0001AF039EF16F087C32AF188C32BF189C3C7
:1039B0002CF18AC32DF18BC32EF18CC32FF18DC353
:1039C00030F18EC331F190C332F191C333F1010173
:1039D000296B3CEC21F0B3EC20F0880E046F130E41
:1039E000056F000E066F000E076FF8EC1FF0000E5B
:1039F000046F040E056F000E066F000E076F04ECD7
:103A000020F00101E80E046F800E056F000E066FB6
:103A1000000E076F24EC20F0060E0C6E00C10BF0B8
:103A2000A7EC07F0070E0C6E01C10BF0A7EC07F036
:103A3000080E0C6E02C10BF0A7EC07F0090E0C6E1D
:103A400003C10BF0A7EC07F004017A0E826FB6EC0D
:103A50000AF004012C0E826FB6EC0AF00401380E55
:103A6000826FB6EC0AF004012C0E826FB6EC0AF0FD
:103A700038EC1BF039EF16F081A8FAEF1DF007A81B
:103A8000B3EF1DF00101800E006F1A0E016F060EDC
:103A9000026F000E036F4BC104F14CC105F14DC123
:103AA00006F14EC107F1F3EC1FF003BFFAEF1DF072
:103AB0006EEC1EF04BC100F14CC101F14DC102F1A1
:103AC0004EC103F1078200EC1FF018C104F119C1C7
:103AD00005F11AC106F11BC107F1F80E006FCD0EFA
:103AE000016F660E026F030E036FF3EC1FF00E0EF4
:103AF0000C6E00C10BF0A7EC07F00F0E0C6E01C1AD
:103B00000BF0A7EC07F0100E0C6E02C10BF0A7EC47
:103B100007F0110E0C6E03C10BF0A7EC07F0078441
:103B20000101EEEC20F057C100F158C101F10794FA
:103B30000A0E0C6E00C10BF0A7EC07F00B0E0C6E1A
:103B400001C10BF0A7EC07F00C0E0C6E02C10BF0DC
:103B5000A7EC07F00D0E0C6E03C10BF0A7EC07F0FD
:103B60000798FAEF1DF007AAFAEF1DF0078401018C
:103B7000EEEC20F057C100F158C101F10794060E98
:103B80000C6E00C10BF0A7EC07F0070E0C6E01C124
:103B90000BF0A7EC07F0080E0C6E02C10BF0A7ECBF
:103BA00007F0090E0C6E03C10BF0A7EC07F00784B9
:103BB00062C100F163C101F164C102F165C103F1A9
:103BC0000794120E0C6E00C10BF0A7EC07F0130E59
:103BD0000C6E01C10BF0A7EC07F0140E0C6E02C1C5
:103BE0000BF0A7EC07F0150E0C6E03C10BF0A7EC61
:103BF00007F0079A0401805181197F0B0BE09EA802
:103C000009D014EE00F081517F0BE126E750812BA3
:103C10000F01AD6E05012F51010A13E081AA21EFBA
:103C20001EF005012F51000A0AE00FB821EF1EF027
:103C30000501306721EF1EF00FB821EF1EF0CFEF26
:103C400027F081B836EF1EF00CEC22F005012F5161
:103C5000020A02E036EF1EF05C2F36EF1EF05BC565
:103C60005CF50501010E306F3C0E316F1AEF0AF062
:103C700018C100F119C101F11AC102F11BC103F110
:103C8000000E046F000E056F010E066F000E076F29
:103C900024EC20F029A163EF1EF02051D8B463EF8B
:103CA0001EF018C100F119C101F11AC102F11BC1C6
:103CB00003F1000E046F000E056F0A0E066F000E72
:103CC000076F24EC20F0120001010451001305518C
:103CD0000113065102130751031312000101186B5F
:103CE000196B1A6B1B6B12002AC182F40401300E8F
:103CF0008227B6EC0AF02BC182F40401300E822731
:103D0000B6EC0AF02CC182F40401300E8227B6EC26
:103D10000AF02DC182F40401300E8227B6EC0AF0BD
:103D20002EC182F40401300E8227B6EC0AF02FC1B6
:103D300082F40401300E8227B6EC0AF030C182F41E
:103D40000401300E8227B6EC0AF031C182F404017E
:103D5000300E8227B6EC0AF032C182F40401300E34
:103D60008227B6EC0AF033C182F40401300E8227B8
:103D7000B6EC0AF012002FC182F40401300E822743
:103D8000B6EC0AF030C182F40401300E8227B6ECA2
:103D90000AF031C182F40401300E8227B6EC0AF039
:103DA00032C182F40401300E8227B6EC0AF033C12E
:103DB00082F40401300E8227B6EC0AF01200060EDF
:103DC000116E060E126E060E136E112EE5EF1EF02A
:103DD000122EE5EF1EF0132EE5EF1EF08B84020E7F
:103DE000116E020E126E020E136E112EF5EF1EF002
:103DF000122EF5EF1EF0132EF5EF1EF08B9412002D
:103E00000101005305E1015303E1025301E1002BDD
:103E1000C3EC1FF0EEEC20F03951006F3A51016F06
:103E2000420E046F4B0E056F000E066F000E076FFB
:103E300004EC20F000C104F101C105F102C106F15A
:103E400003C107F118C100F119C101F11AC102F152
:103E50001BC103F107B231EF1FF0F8EC1FF033EF95
:103E60001FF0F3EC1FF000C118F101C119F102C1FC
:103E70001AF103C11BF11200EEEC20F059C100F160
:103E80005AC101F1060EBEEC07F0E8CF04F1070EAF
:103E9000BEEC07F0E8CF05F1080EBEEC07F0E8CF66
:103EA00006F1090EBEEC07F0E8CF07F1F3EC1FF0C6
:103EB00000C124F101C125F102C126F103C127F19E
:103EC000290E046F000E056F000E066F000E076FBF
:103ED00004EC20F0EE0E046F430E056F000E066F2B
:103EE000000E076FF8EC1FF024C104F125C105F1A5
:103EF00026C106F127C107F104EC20F000C11CF136
:103F000001C11DF102C11EF103C11FF1120EBEEC71
:103F100007F0E8CF04F1130EBEEC07F0E8CF05F18F
:103F2000140EBEEC07F0E8CF06F1150EBEEC07F05C
:103F3000E8CF07F10D0E006F000E016F000E026F4B
:103F4000000E036F04EC20F0180E046F000E056FD6
:103F5000000E066F000E076F24EC20F01CC104F168
:103F60001DC105F11EC106F11FC107F1F8EC1FF0DC
:103F70006A0E046F2A0E056F000E066F000E076FA3
:103F8000F3EC1FF01200BF0EFA6E200E3A6F396B81
:103F9000D8900037013702370337D8B0D4EF1FF07D
:103FA0003A2FC9EF1FF039073A070353D8B412006C
:103FB0000331070B80093F6F03390F0B010F396F76
:103FC00080EC5FF0406F390580EC5FF0405D405F52
:103FD000396B3F33D8B0392739333FA9E9EF1FF0A8
:103FE000405139271200010113EC21F0D8B0120022
:103FF000010103510719346FD6EC20F0D890075116
:10400000031934AF800F12000101346BFAEC20F079
:10401000D8A010EC21F0D8B01200E5EC20F0EEECC6
:1040200020F01F0E366F26EC21F00B35D8B0D6EC01
:1040300020F0D8A00335D8B01200362F13EF20F0AF
:1040400034B1FDEC20F012000101346B0451051174
:10405000061107110008D8A0FAEC20F0D8A010EC47
:1040600021F0D8B01200086B096B0A6B0B6B26ECC1
:1040700021F01F0E366F26EC21F007510B5DD8A4FE
:104080004EEF20F006510A5DD8A44EEF20F0055106
:10409000095DD8A44EEF20F00451085DD8A061EF6F
:1040A00020F00451085F0551D8A0053D095F065175
:1040B000D8A0063D0A5F0751D8A0073D0B5FD890F6
:1040C0000081362F3BEF20F034B1FDEC20F0346B53
:1040D000FAEC20F0D8902AEC21F007510B5DD8A41F
:1040E0007EEF20F006510A5DD8A47EEF20F0055146
:1040F000095DD8A47EEF20F00451085DD8A08DEFB3
:1041000020F0003F8DEF20F0013F8DEF20F0023FC7
:104110008DEF20F0032BD8B4120034B1FDEC20F069
:1041200012000101346BFAEC20F0D8B012002FEC31
:1041300021F0200E366F003701370237033711EEBA
:1041400033F00A0E376FE7360A0EE75CD8B0E76E39
:10415000E552372FA3EF20F0362F9BEF20F034B13C
:104160002981D890120001010A0E346F200E366F9B
:1041700011EE29F03451376F0A0ED890E652D8B0BC
:10418000E726E732372FBEEF20F003330233013347
:104190000033362FB8EF20F0E750FF0FD8A00335DB
:1041A000D8B0120029B1FDEC20F012000451002714
:1041B0000551D8B0053D01270651D8B0063D02276C
:1041C0000751D8B0073D032712000051086F015175
:1041D000096F02510A6F03510B6F12000101006B4E
:1041E000016B026B036B12000101046B056B066B24
:1041F000076B12000335D8A012000351800B001F7B
:10420000011F021F031F003F0DEF21F0013F0DEFC3
:1042100021F0023F0DEF21F0032B342B0325120078
:104220000735D8A012000751800B041F051F061F79
:10423000071F043F23EF21F0053F23EF21F0063F46
:1042400023EF21F0072B342B07251200003701370D
:1042500002370337083709370A370B3712000101D5
:10426000296B2A6B2B6B2C6B2D6B2E6B2F6B306B92
:10427000316B326B336B120001012A510F0B2A6F25
:104280002B510F0B2B6F2C510F0B2C6F2D510F0B34
:104290002D6F2E510F0B2E6F2F510F0B2F6F305193
:1042A0000F0B306F31510F0B316F32510F0B326FDB
:1042B00033510F0B336F12008984000EC76E220E2C
:1042C000C66E9E96C69E000EC96EFF0E9EB602D0AA
:1042D000E82EFCD79E96C69E000EC96EFF0E9EB6B7
:1042E00002D0E82EFCD7C9CFABF59E96C69E000E35
:1042F000C96EFF0E9EB602D0E82EFCD7C9CFACF532
:104300009E96C69E000EC96EFF0E9EB602D0E82E87
:10431000FCD7C9CFADF59E96C69E000EC96EFF0EA6
:104320009EB602D0E82EFCD7C9CFAEF59E96C69EAB
:10433000000EC96EFF0E9EB602D0E82EFCD7C9CF84
:10434000AFF59E96C69E000EC96EFF0E9EB602D0B9
:10435000E82EFCD7C9CFB0F59E96C69E000EC96E5A
:10436000FF0E9EB602D0E82EFCD7C9CFB1F58994D6
:104370000FEC24F012008984000EC76E220EC66E68
:104380009E96C69E800EC96EFF0E9EB602D0E82E87
:10439000FCD79E96C69EABC5C9FFFF0E9EB602D047
:1043A000E82EFCD79E96C69EACC5C9FFFF0E9EB6F2
:1043B00002D0E82EFCD79E96C69EADC5C9FFFF0E63
:1043C0009EB602D0E82EFCD79E96C69EAEC5C9FF0B
:1043D000FF0E9EB602D0E82EFCD79E96C69EAFC5B5
:1043E000C9FFFF0E9EB602D0E82EFCD79E96C69E51
:1043F000B0C5C9FFFF0E9EB602D0E82EFCD79E9630
:10440000C69EB1C5C9FFFF0E9EB602D0E82EFCD7EE
:1044100089940FEC24F012008984000EC76E220EDE
:10442000C66E9E96C69E070EC96EFF0E9EB602D041
:10443000E82EFCD79E96C69E000EC96EFF0E9EB655
:1044400002D0E82EFCD7C9CFABF59E96C69E000ED3
:10445000C96EFF0E9EB602D0E82EFCD7C9CFACF5D0
:104460009E96C69E000EC96EFF0E9EB602D0E82E26
:10447000FCD7C9CFADF59E96C69E000EC96EFF0E45
:104480009EB602D0E82EFCD7C9CFAEF589940FECCA
:1044900024F08984000EC76E220EC66E9E96C69EBC
:1044A0000F0EC96EFF0E9EB602D0E82EFCD79E9668
:1044B000C69E000EC96EFF0E9EB602D0E82EFCD737
:1044C000C9CFB3F589940FEC24F012008984000E53
:1044D000C76E220EC66E9E96C69E870EC96EFF0ED2
:1044E0009EB602D0E82EFCD79E96C69EABC5C9FFED
:1044F000FF0E9EB602D0E82EFCD79E96C69EACC597
:10450000C9FFFF0E9EB602D0E82EFCD79E96C69E2F
:10451000ADC5C9FFFF0E9EB602D0E82EFCD79E9611
:10452000C69EAEC5C9FFFF0E9EB602D0E82EFCD7D0
:1045300089940FEC24F089849E96C69E8F0EC96ED6
:10454000FF0E9EB602D0E82EFCD79E96C69EB3C53F
:10455000C9FFFF0E9EB602D0E82EFCD789940FEC5F
:1045600024F012008984000EC76E220EC66E9E963D
:10457000C69E870EC96EFF0E9EB602D0E82EFCD7EF
:104580009E96C69E000EC96EFF0E9EB602D0E82E05
:10459000FCD79E96C69E800EC96EFF0E9EB602D0B8
:1045A000E82EFCD79E96C69E800EC96EFF0E9EB664
:1045B00002D0E82EFCD79E96C69E800EC96EFF0ED6
:1045C0009EB602D0E82EFCD789940FEC24F08984A3
:1045D0009E96C69E8F0EC96EFF0E9EB602D0E82E26
:1045E000FCD79E96C69E010EC96EFF0E9EB602D0E7
:1045F000E82EFCD789940FEC24F012008984000E79
:10460000C76E220EC66E9E96C69E870EC96EFF0EA0
:104610009EB602D0E82EFCD79E96C69E000EC96EAE
:10462000FF0E9EB602D0E82EFCD79E96C69E000EC8
:10463000C96EFF0E9EB602D0E82EFCD79E96C69E8F
:10464000800EC96EFF0E9EB602D0E82EFCD79E9655
:10465000C69E800EC96EFF0E9EB602D0E82EFCD715
:1046600089940FEC24F089849E96C69E8F0EC96EA5
:10467000FF0E9EB602D0E82EFCD79E96C69E010E77
:10468000C96EFF0E9EB602D0E82EFCD789940FECBF
:1046900024F012008984000EC76E220EC66E9E960C
:1046A000C69E8F0EC96EFF0E9EB602D0E82EFCD7B6
:1046B0000FEC24F09E96C69E810EC96EFF0E9EB62C
:1046C00002D0E82EFCD789940FEC24F08984000EE8
:1046D000C76E220EC66E9E96C69E8F0EC96EFF0EC8
:1046E0009EB602D0E82EFCD70FEC24F09E96C69E14
:1046F000010EC96EFF0E9EB602D0E82EFCD789943B
:104700000FEC24F089849E96C69E910EC96EFF0E12
:104710009EB602D0E82EFCD70FEC24F09E96C69EE3
:10472000A50EC96EFF0E9EB602D0E82EFCD7899466
:104730000FEC24F012008984000EC76E220EC66EA4
:104740009E96C69E8F0EC96EFF0E9EB602D0E82EB4
:10475000FCD70FEC24F09E96C69E810EC96EFF0E0C
:104760009EB602D0E82EFCD789940FEC24F01200FC
:104770008984000EC76E220EC66E9E96C69E8F0E50
:10478000C96EFF0E9EB602D0E82EFCD70FEC24F0C7
:104790009E96C69E010EC96EFF0E9EB602D0E82EF2
:1047A000FCD789940FEC24F012008984000EC76EA8
:1047B000220EC66E9E96C69E910EC96EFF0E9EB6C6
:1047C00002D0E82EFCD70FEC24F09E96C69EA50ED4
:1047D000C96EFF0E9EB602D0E82EFCD789940FEC6E
:1047E00024F012008984000EC76E220EC66E9E96BB
:1047F000C69E910EC96EFF0E9EB602D0E82EFCD763
:104800000FEC24F09E96C69E000EC96EFF0E9EB65B
:1048100002D0E82EFCD789940FEC24F01200050E8C
:10482000E82EFED712000501256B266B276B286B3F
:10483000899A400EC76E200EC66E9E96C69E030EC7
:10484000C96EFF0E9EB602D0E82EFCD79E96C69E7D
:1048500027C5C9FFFF0E9EB602D0E82EFCD79E9654
:10486000C69E26C5C9FFFF0E9EB602D0E82EFCD715
:104870009E96C69E25C5C9FFFF0E9EB602D0E82EA5
:10488000FCD79E96C69EC952FF0E9EB602D0E82E59
:10489000FCD7898A0F01C950FF0A01E11200050106
:1048A0002E51130A05E005012E51170A0CE01200E3
:1048B0000501F00E256FFF0E266F0F0E276F000EFD
:1048C000286F6CEF24F00501F00E256FFF0E266FA8
:1048D000FF0E276F000E286F899A400EC76E200EBC
:1048E000C66E9E96C69E030EC96EFF0E9EB602D081
:1048F000E82EFCD79E96C69E27C5C9FFFF0E9EB622
:1049000002D0E82EFCD79E96C69E26C5C9FFFF0E94
:104910009EB602D0E82EFCD79E96C69E25C5C9FF3E
:10492000FF0E9EB602D0E82EFCD79E96C69EC952B8
:10493000FF0E9EB602D0E82EFCD7898A0F01C9501F
:10494000FF0A1DE005012E51130A05E005012E5155
:10495000170A0BE012000501000E256F000E266FEE
:10496000100E276F000E286F12000501000E256F34
:10497000000E266F000E276F010E286F1200050132
:10498000256B266B276B286B05012E51130A05E05A
:1049900005012E51170A0CE012000501000E216FCF
:1049A000000E226F080E236F000E246FE1EF24F03B
:1049B0000501000E216F000E226F800E236F000E86
:1049C000246F21C500F122C501F123C502F124C5E0
:1049D00003F125C504F126C505F127C506F128C553
:1049E00007F164EC1EF000C125F501C126F502C1F6
:1049F00027F503C128F5899A400EC76E200EC66EB2
:104A00009E96C69E030EC96EFF0E9EB602D0E82E7D
:104A1000FCD79E96C69E27C5C9FFFF0E9EB602D044
:104A2000E82EFCD79E96C69E26C5C9FFFF0E9EB6F1
:104A300002D0E82EFCD79E96C69E25C5C9FFFF0E64
:104A40009EB602D0E82EFCD79E96C69EC952FF0E97
:104A50009EB602D0E82EFCD7898AC950FF0A08E129
:104A600004C125F505C126F506C127F507C128F5BE
:104A7000D890050124332333223321332151F00B05
:104A8000216F21674BEF25F022674BEF25F023675D
:104A90004BEF25F02467E1EF24F00501100E2527E8
:104AA000E86A2623E86A2723E86A28231200E86ACE
:104AB00005012E51130A06E005012E51170A0BE0DD
:104AC000020E120005012851000A03E12751F00BE4
:104AD00007E0010E120005012851000A01E0010E55
:104AE000120029C500F12AC501F12BC502F12CC520
:104AF00003F125C504F126C505F127C506F128C532
:104B000007F1F3EC1FF003BF120057EC25F0D8A417
:104B1000E9EF25F0899A400EC76E200EC66E9E966C
:104B2000C69E060EC96EFF0E9EB602D0E82EFCD7BA
:104B3000898A899A9E96C69E020EC96EFF0E9EB6FF
:104B400002D0E82EFCD79E96C69E27C5C9FFFF0E51
:104B50009EB602D0E82EFCD79E96C69E26C5C9FFFB
:104B6000FF0E9EB602D0E82EFCD79E96C69E25C5A7
:104B7000C9FFFF0E9EB602D0E82EFCD79E96C69EB9
:104B8000000EC96EFF0E9EB602D0E82EFCD7898AB1
:104B9000899A9E96C69E050EC96EFF0E9EB602D0DD
:104BA000E82EFCD79E96C69EC952FF0E9EB602D036
:104BB000E82EFCD7C9B0D2EF25F0898A0501100E86
:104BC0002527E86A2623E86A2723E86A282371EF65
:104BD00025F01200899A400EC76E200EC66E9E9672
:104BE000C69E060EC96EFF0E9EB602D0E82EFCD7FA
:104BF000898A899A9E96C69EC70EC96EFF0E9EB67A
:104C000002D0E82EFCD7898A0501256B266B276B1D
:104C1000286B1200899A400EC76E200EC66E9E96B3
:104C2000C69E050EC96EFF0E9EB602D0E82EFCD7BA
:104C30009E96C69EC952FF0E9EB602D0E82EFCD7A5
:104C4000C9CF33F5898A1200899A400EC76E200EAB
:104C5000C66E9E96C69EB90EC96EFF0E9EB602D057
:104C6000E82EFCD7898A1200899A400EC76E200E62
:104C7000C66E9E96C69EAB0EC96EFF0E9EB602D045
:104C8000E82EFCD7898AFF0EE82EFED7120057ECDB
:104C900025F0D8A41200899A400EC76E200EC66E69
:104CA0009E96C69E030EC96EFF0E9EB602D0E82EDB
:104CB000FCD79E96C69E27C5C9FFFF0E9EB602D0A2
:104CC000E82EFCD79E96C69E26C5C9FFFF0E9EB64F
:104CD00002D0E82EFCD79E96C69E25C5C9FFFF0EC2
:104CE0009EB602D0E82EFCD79E96C69EC952FF0EF5
:104CF0009EB602D0E82EFCD7898A0F01C950FF0A60
:104D0000D8A442EF27F00501FE0E336F5CEC21F0D2
:104D1000ABC534F5ACC535F5ADC536F5AEC537F523
:104D2000AFC538F5B0C539F5B1C53AF50784B6C198
:104D300066F1B7C167F1B8C168F1B9C169F14BC19A
:104D40004FF14CC150F14DC151F14EC152F157C11B
:104D500059F158C15AF163EC16F000C13BF501C19D
:104D60003CF502C13DF503C13EF505015D67C0EFAD
:104D700026F05E67C0EF26F05F67C0EF26F0606741
:104D8000C4EF26F0D1EF26F05DC504F15EC505F154
:104D90005FC506F160C507F1F3EC1FF003BF42EFFA
:104DA00027F059C13FF55AC140F5B5C541F5B6C523
:104DB00042F507940501110E326F899A400EC76EB5
:104DC000200EC66E9E96C69E060EC96EFF0E9EB63D
:104DD00002D0E82EFCD7898A899A9E96C69E020E3A
:104DE000C96EFF0E9EB602D0E82EFCD79E96C69ED8
:104DF00027C5C9FFFF0E9EB602D0E82EFCD79E96AF
:104E0000C69E26C5C9FFFF0E9EB602D0E82EFCD76F
:104E10009E96C69E25C5C9FFFF0E9EB602D0E82EFF
:104E2000FCD725EE33F0322F02D022EF27F09E96EA
:104E3000C69EDECFC9FFFF0E9EB602D0E82EFCD77D
:104E400013EF27F0898A899A9E96C69E050EC96E31
:104E5000FF0E9EB602D0E82EFCD79E96C69EC95283
:104E6000FF0E9EB602D0E82EFCD7C9B02DEF27F07A
:104E7000898A0501100E2527E86A2623E86A272378
:104E8000E86A2823120021C500F122C501F123C5DB
:104E900002F124C503F1899A400EC76E200EC66E3A
:104EA0009E96C69E0B0EC96EFF0E9EB602D0E82ED1
:104EB000FCD79E96C69E02C1C9FFFF0E9EB602D0C9
:104EC000E82EFCD79E96C69E01C1C9FFFF0E9EB676
:104ED00002D0E82EFCD79E96C69E00C1C9FFFF0EE9
:104EE0009EB602D0E82EFCD79E96C69EC952FF0EF3
:104EF0009EB602D0E82EFCD725EE33F00501100E49
:104F0000326F9E96C69EC952FF0E9EB602D0E82E04
:104F1000FCD7C9CFDEFF322F81EF27F0898A12003C
:104F2000899A400EC76E200EC66E9E96C69E900E43
:104F3000C96EFF0E9EB602D0E82EFCD79E96C69E86
:104F4000000EC96EFF0E9EB602D0E82EFCD79E96CC
:104F5000C69E000EC96EFF0E9EB602D0E82EFCD78C
:104F60009E96C69E000EC96EFF0E9EB602D0E82E1B
:104F7000FCD79E96C69EC952FF0E9EB602D0E82E62
:104F8000FCD7C9CF2DF59E96C69EC952FF0E9EB680
:104F900002D0E82EFCD7C9CF2EF5898A1200DFECAB
:104FA0001EF0B5C5E8FFD70802E3DFEC1EF0B5C57B
:104FB000E8FFC80802E3DFEC1EF0B5C5E8FFB9085A
:104FC00002E3DFEC1EF0B5C5E8FFAA0802E3DFEC60
:104FD0001EF0B5C5E8FF9B0802E3DFEC1EF00CEC09
:104FE00022F024EC26F0F29CF29E8B94C69AC2909A
:104FF0009482948C720ED36ED3A4FED789968A9035
:105000009390FF0EE8CF00F0E82EFED7002EFCD7DD
:105010008150F294F29A9E909D909E929D92F29869
:0C502000F292F290F286F28E0300FF0084
:10BF0000E844F926000C160C2B0C3F0C520C640C68
:10BF1000760C860C960CA50CB30CC10CCF0CDC0C6B
:06BF2000E80CF40C000C1B
:00000001FF
